:020000040000FA
:02000000F128E5
:080008008C00030E8D00831231
:100010000B1D4528051C0E28A90AA919A903A91B0F
:10002000A9012908063A03190E16073A03190E12F8
:100030008E1834280E1E34288E1493010E1C3C2872
:1000400094011C0895001D0896001E0897002108C1
:100050009A001F0898002008990022089B00C830C9
:1000600092000E100E1545288E1C3C280E1A3C28B6
:100070008E101308E23E4821920B4228C8309200AD
:100080008D210E15930F45284F210B110D0E830066
:100090008C0E0C0E090082078234A834A8348C34EC
:1000A000863481342D344434433446343734373441
:1000B0002D344F3472346134203430342E3439349A
:1000C00061342D34FF344E347934E1347234693480
:1000D000203469346434F5342034FF345434E93442
:1000E0006C346934203469346434F5342034203479
:1000F000FF342D342D342D342D342D342D342D3426
:100100002D342D34FF3448346534743466346F3400
:100110002034203420342034FF344B3465346434AC
:10012000643420342034203420342034FF345334D9
:100130007A346534723464346134203420342034A9
:10014000FF3443347334753474346F34723474341C
:100150006F346B34FF34503465346E34743465342A
:100160006B34203420342034FF3453347A346F34E9
:100170006D3462346134743420342034FF345634A6
:1001800061347334613472346E34613470342034C9
:10019000FF3482072D342D342D344A3461346E34CB
:1001A0004634653462344D346134723441347034D1
:1001B00072344D3461346A344A3475346E344A349E
:1001C00075346C3441347534673453347A3465345F
:1001D0004F346B3474344E346F3476344434653475
:1001E00063348316033081000330850000308600BD
:1001F0008312850186018E019301C830920094011B
:10020000950196019A019901013098009700A0305C
:100210008B00022264000E1D0A290130E8216400CF
:100220000E1D0F290E11172116210F2908008030ED
:10023000E821160811223A30E921150811223A3036
:10024000E921140811222030E92122301B1A17302D
:1002500000222030E921C030E8211A0D8F000F0D57
:10026000FC391A078F0003100F0D2D3E002220309D
:10027000E921170811222E30E9212030E921180840
:1002800024222030E921190811222030E921080018
:10029000A00C9F0C9E0C9D0C9C0CA20C08001F0D2A
:1002A000A00D1E0D1F0D0739A1009F0C9F0C1F30C4
:1002B0009F059E0C3F309E051D0C9C0CA20C9C0CB7
:1002C000A20C7F309C059D0C9D0C3F309D0523307A
:1002D000840096211C082306031D81291D0824067D
:1002E000031D81291E082506031D81291F082606D6
:1002F000031D812920082706031D81298E150E1450
:1003000008001C08A3001D08A4001E08A5001F0863
:10031000A6002008A7008E11080014308400D921FF
:1003200060300006031D08008001840AD921603076
:100330000006031D08008001840AD921243000062C
:10034000031D08008001840AD921840A840A840AD2
:10035000800A013080198000840384030830000281
:1003600000080318F93E0139313E8F000008023AB7
:10037000031DC72930308F00840A00088403133915
:100380000319C729123A0319C72929308F0084039A
:100390000F080006031D080001308000840AD921DF
:1003A0000008133A031D080001308000840AD92197
:1003B0000800800A06300007831880000430860099
:1003C0008614060D8610861486100318E02908008E
:1003D0008E179000DE2183160030860083121008ED
:1003E000F921100EF9218E138316F0308600831246
:1003F0000800F0398E1F0838860086148610080021
:100400009100032A910111084B20FF3A03190800BB
:10041000FF3A90008E17901F8E137F39E921910AC1
:10042000032A9100110E152211080F39063E831878
:10043000073E2A3EE92907399100910711087920E2
:10044000E921110A7920E9299100FA30111A91075E
:100450000310110D91071108C920E921910A110813
:0A046000C920E921110AC920E92989
:02400E00F53F7C
:00000001FF
